:100000009128A0003F200C080D0403198C2886209D
:1000100084132008800664000D280E288C0A03191A
:100020008D0F0B2880068C288F0022088400200961
:10003000402084138F0803198C28F03091000E089B
:1000400080389000F03091030319910003198F0359
:1000500003198C282B28552003010C1820088E1F0B
:1000600020088E0803190301900F382880061F28E6
:100070003928000022284320FF3A80054028FF3A13
:10008000841780058C28940006309419053084006C
:1000900000308A001408073982070134023404341E
:1000A000083410342034403480340D080C04031913
:1000B0008C0A80300C1A8D060C198D068C188D0652
:1000C0000D0D8C0D8D0D8C288F018E00FF308E074D
:1000D000031C8F07031C8C2803308D00DF30722037
:1000E00066288D01E83E8C008D09FC30031C7B28BE
:1000F0008C07031878288C0764008D0F78280C185B
:1001000081288C1C85280000852808008C098D0911
:100110008C0A03198D0A08008313031383126400E9
:1001200008008316850103308600831205118316AB
:1001300005118312851183168511831227083B2030
:1001400028083B2029083B202A083B202B083B207D
:100150002C083B200130AD00640008302D0203184C
:10016000C92805158316051183128511831685117B
:100170008312DB20323064200511831605118312AF
:100180008515831685118312DB2032306420AD0F74
:10019000AC2885118316851183129630A7009630FE
:1001A000A8009630A9009630AA009630AB00963091
:1001B000AC00F020CD2824088C0025088D005520A7
:1001C0000C08A4000D08A5005F302405A60005302A
:1001D000A2001030A00026088E0004301420080071
:1001E0000130AE00640015302E02031825292708BF
:1001F0008C008D01063084000430012028088C001A
:100200008D01063084000830012029088C008D0102
:1002100006308400803001202A088C008D010630D1
:100220008400403001202B088C008D0106308400B2
:10023000203001202C088C008D0106308400103005
:0C02400001200C306420AE0FF2280800F2
:02400E00F53F7C
:00000001FF
